Archive member included       because of file (symbol)

C:/agb/lib/libagbsyscall.a(AgbSysCpuFastSet.o)
                              sub.o (CpuFastSet)
C:/agb/lib/libagbsyscall.a(AgbSysCpuSet.o)
                              MultiSio.o (CpuSet)
C:/agb/lib/libagbsyscall.a(AgbSysIntrWait.o)
                              loader_main.o (IntrWait)
C:/agb/lib/libagbsyscall.a(AgbSysRegisterRamReset.o)
                              loader_main.o (RegisterRamReset)
C:/agb/lib/libagbsyscall.a(AgbSysVBlankIntrWait.o)
                              loader_main.o (VBlankIntrWait)
C:\PROGRA~1\CYGNUS\THUMBELF-000512\H-I686-CYGWIN32\BIN/../lib/gcc-lib/thumb-elf/2.9-arm-000512/libgcc.a(_call_via_rX.o)
                              loader_main.o (_call_via_r0)

Allocating common symbols
Common symbol       size              file

S32ml               0x18              Sio32MultiLoad.o
UsrSendBuf          0x10              bss.o
BurstLoad           0x4               loader_main.o
IntrTableBuf        0x34              intr_table.o
Cont                0x4               bss.o
SioFlagsBak         0x4               bss.o
RecvLoadCounter     0x4               loader_main.o
IntrFuncBuf         0x100             MultiSio.o
Trg                 0x4               bss.o
SioFlags            0x4               bss.o
SioState            0x4               bss.o
SioStartFlag        0x4               bss.o
LoadCounterp        0x4               loader_main.o
IntrMainBuf         0x400             bss.o
UsrRecvBuf          0x40              bss.o
Ms                  0x158             MultiSio.o
OamBak              0x400             bss.o
ProgressCounter     0x4               loader_main.o
RecvFuncBuf         0x40              MultiSio.o
BgBak               0x800             bss.o

Memory Configuration

Name             Origin             Length             Attributes
*default*        0x00000000         0xffffffff

Linker script and memory map

LOAD crt0_loader.o
LOAD intr_main.o
LOAD MultiSioAsm.o
LOAD loader_main.o
LOAD sub.o
LOAD intr_table.o
LOAD bss.o
LOAD data.o
LOAD load_table_dest.o
LOAD MultiSio.o
LOAD Sio32MultiLoad.o
LOAD C:/agb/lib/libagbsyscall.a
LOAD C:/agb/lib/libisagbprn.a
LOAD C:\PROGRA~1\CYGNUS\THUMBELF-000512\H-I686-CYGWIN32\BIN/../lib/gcc-lib/thumb-elf/2.9-arm-000512/libgcc.a
LOAD C:\PROGRA~1\CYGNUS\THUMBELF-000512\H-I686-CYGWIN32\BIN/../lib/gcc-lib/thumb-elf/2.9-arm-000512/../../../../thumb-elf/lib/libg.a
LOAD C:\PROGRA~1\CYGNUS\THUMBELF-000512\H-I686-CYGWIN32\BIN/../lib/gcc-lib/thumb-elf/2.9-arm-000512/../../../../thumb-elf/lib/libc.a
LOAD C:\PROGRA~1\CYGNUS\THUMBELF-000512\H-I686-CYGWIN32\BIN/../lib/gcc-lib/thumb-elf/2.9-arm-000512/libgcc.a
Address of section .text set to 0x2030000
Address of section .bss set to 0x3000000
                0x00008000                .=0x8000

.interp
 *(.interp)

.hash
 *(.hash)

.dynsym
 *(.dynsym)

.dynstr
 *(.dynstr)

.gnu.version
 *(.gnu.version)

.gnu.version_d
 *(.gnu.version_d)

.gnu.version_r
 *(.gnu.version_r)

.rel.text
 *(.rel.text)
 *(.rel.text.*)
 *(.rel.gnu.linkonce.t*)

.rela.text
 *(.rela.text)
 *(.rela.text.*)
 *(.rela.gnu.linkonce.t*)

.rel.data
 *(.rel.data)
 *(.rel.data.*)
 *(.rel.gnu.linkonce.d*)

.rela.data
 *(.rela.data)
 *(.rela.data.*)
 *(.rela.gnu.linkonce.d*)

.rel.rodata
 *(.rel.rodata)
 *(.rel.rodata.*)
 *(.rel.gnu.linkonce.r*)

.rela.rodata
 *(.rela.rodata)
 *(.rela.rodata.*)
 *(.rela.gnu.linkonce.r*)

.rel.got
 *(.rel.got)

.rela.got
 *(.rela.got)

.rel.ctors
 *(.rel.ctors)

.rela.ctors
 *(.rela.ctors)

.rel.dtors
 *(.rel.dtors)

.rela.dtors
 *(.rela.dtors)

.rel.init
 *(.rel.init)

.rela.init
 *(.rela.init)

.rel.fini
 *(.rel.fini)

.rela.fini
 *(.rela.fini)

.rel.bss
 *(.rel.bss)

.rela.bss
 *(.rela.bss)

.rel.plt
 *(.rel.plt)

.rela.plt
 *(.rela.plt)

.init
 *(.init)

.plt
 *(.plt)

.text           0x02030000     0x1034
 *(.text)
 .text          0x02030000       0x48 crt0_loader.o
                0x02030000                _start
                0x02030000                start_vector
 .text          0x02030048       0xf0 intr_main.o
                0x02030048                intr_main
 .text          0x02030138       0x40 MultiSioAsm.o
                0x02030138                MultiSioRecvBufChange
 .text          0x02030178      0x4d0 loader_main.o
                0x02030178                LoaderMain
 .text          0x02030648       0xfc sub.o
                0x020306b0                IntrDummy
                0x02030648                VBlankIntr
                0x020306e4                BgScSet
                0x020306b4                KeyRead
                0x0203070c                Data2BgSc
 .text          0x02030744      0x540 MultiSio.o
                0x02030bb0                MultiSioIntr
                0x02030744                MultiSioInit
                0x02030880                MultiSioMain
                0x02030a08                MultiSioRecvDataCheck
                0x02030830                MultiSioStop
                0x02030b78                MultiSioVSync
                0x02030970                MultiSioSendDataSet
                0x02030818                MultiSioStart
 .text          0x02030c84      0x358 Sio32MultiLoad.o
                0x02030c84                Sio32MultiLoadInit
                0x02030d34                Sio32MultiLoadMain
                0x02030f14                Sio32MultiLoadIntr
 .text          0x02030fdc        0x4 C:/agb/lib/libagbsyscall.a(AgbSysCpuFastSet.o)
                0x02030fdc                CpuFastSet
 .text          0x02030fe0        0x4 C:/agb/lib/libagbsyscall.a(AgbSysCpuSet.o)
                0x02030fe0                CpuSet
 .text          0x02030fe4        0x8 C:/agb/lib/libagbsyscall.a(AgbSysIntrWait.o)
                0x02030fe4                IntrWait
 .text          0x02030fec        0x4 C:/agb/lib/libagbsyscall.a(AgbSysRegisterRamReset.o)
                0x02030fec                RegisterRamReset
 .text          0x02030ff0        0x8 C:/agb/lib/libagbsyscall.a(AgbSysVBlankIntrWait.o)
                0x02030ff0                VBlankIntrWait
 .text          0x02030ff8       0x3c C:\PROGRA~1\CYGNUS\THUMBELF-000512\H-I686-CYGWIN32\BIN/../lib/gcc-lib/thumb-elf/2.9-arm-000512/libgcc.a(_call_via_rX.o)
                0x02031000                _call_via_r2
                0x02031010                _call_via_r6
                0x0203100c                _call_via_r5
                0x02031004                _call_via_r3
                0x02031024                _call_via_fp
                0x02031018                _call_via_r8
                0x02031014                _call_via_r7
                0x02030ff8                _call_via_r0
                0x02031020                _call_via_sl
                0x0203102c                _call_via_sp
                0x0203101c                _call_via_r9
                0x02031008                _call_via_r4
                0x02030ffc                _call_via_r1
                0x02031028                _call_via_ip
                0x02031030                _call_via_lr
 *(.text.*)
 *(.stub)
 *(.gnu.warning)
 *(.gnu.linkonce.t*)
 *(.glue_7t)
 *(.glue_7)
                0x02031034                _etext=.
                0x02031034                PROVIDE (etext, .)

.fini
 *(.fini)

.rodata         0x02031034     0x23c8
 *(.rodata)
 .rodata        0x02031034       0x2c loader_main.o
 .rodata        0x02031060       0x34 intr_table.o
                0x02031060                IntrTable
 .rodata        0x02031094     0x2320 data.o
                0x02031594                OamData_Sample
                0x020315b4                PlttData_Sample
                0x020317b4                CharData_Sample
                0x02031094                BgScData_Sample
 .rodata        0x020333b4       0x10 load_table_dest.o
                0x020333b4                LoadTable
 .rodata        0x020333c4       0x20 MultiSio.o
 .rodata        0x020333e4       0x18 Sio32MultiLoad.o
 *(.rodata.*)
 *(.gnu.linkonce.r*)

.rodata1
 *(.rodata1)
                0x020334fc                .=(ALIGN(0x100)+(.&0xff))

.data           0x020334fc        0x0
 *(.data)
 *(.data.*)
 *(.gnu.linkonce.d*)

.data1
 *(.data1)

.ctors
 EXCLUDE_FILE ( *crtend.o )*(.ctors)
 *(SORT(.ctors.*))
 *crtend(.ctors)

.dtors
 EXCLUDE_FILE ( *crtend.o )*(.dtors)
 *(SORT(.dtors.*))
 *crtend.o(.dtors)

.got
 *(.got.plt)
 *(.got)

.dynamic
 *(.dynamic)

.sdata
 *(.sdata)
 *(.sdata.*)
                0x020334fc                _edata=.
                0x020334fc                PROVIDE (edata, .)
                0x020334fc                __bss_start=.
                0x020334fc                __bss_start__=.

.sbss
 *(.sbss)
 *(.scommon)

.bss            0x03000000     0x1378
 *(.dynbss)
 *(.bss)
 *(.bss.*)
 *(COMMON)
 COMMON         0x03000000       0x10 loader_main.o
                                  0x0 (size before relaxing)
                0x03000000                BurstLoad
                0x03000004                RecvLoadCounter
                0x03000008                LoadCounterp
                0x0300000c                ProgressCounter
 COMMON         0x03000010       0x34 intr_table.o
                                  0x0 (size before relaxing)
                0x03000010                IntrTableBuf
 *fill*         0x03000044        0xc
 COMMON         0x03000050     0x1070 bss.o
                                  0x0 (size before relaxing)
                0x03000050                UsrSendBuf
                0x03000060                Cont
                0x03000064                SioFlagsBak
                0x03000068                Trg
                0x0300006c                SioFlags
                0x03000070                SioState
                0x03000074                SioStartFlag
                0x03000080                IntrMainBuf
                0x03000480                UsrRecvBuf
                0x030004c0                OamBak
                0x030008c0                BgBak
 COMMON         0x030010c0      0x2a0 MultiSio.o
                                  0x0 (size before relaxing)
                0x030010c0                IntrFuncBuf
                0x030011c0                Ms
                0x03001320                RecvFuncBuf
 COMMON         0x03001360       0x18 Sio32MultiLoad.o
                                  0x0 (size before relaxing)
                0x03001360                S32ml
                0x03001378                .=ALIGN(0x4)
                0x03001378                .=ALIGN(0x4)
                0x03001378                _end=.
                0x03001378                _bss_end__=.
                0x03001378                __bss_end__=.
                0x03001378                PROVIDE (end, .)

.stab
 *(.stab)

.stabstr
 *(.stabstr)

.stab.excl
 *(.stab.excl)

.stab.exclstr
 *(.stab.exclstr)

.stab.index
 *(.stab.index)

.stab.indexstr
 *(.stab.indexstr)

.comment
 *(.comment)

.debug
 *(.debug)

.line
 *(.line)

.debug_srcinfo
 *(.debug_srcinfo)

.debug_sfnames
 *(.debug_sfnames)

.debug_aranges  0x00000000       0x80
 *(.debug_aranges)
 .debug_aranges
                0x00000000       0x20 loader_main.o
 .debug_aranges
                0x00000020       0x20 sub.o
 .debug_aranges
                0x00000040       0x20 MultiSio.o
 .debug_aranges
                0x00000060       0x20 Sio32MultiLoad.o

.debug_pubnames
                0x00000000      0x344
 *(.debug_pubnames)
 .debug_pubnames
                0x00000000       0x68 loader_main.o
 .debug_pubnames
                0x00000068       0x55 sub.o
 .debug_pubnames
                0x000000bd       0x31 intr_table.o
 .debug_pubnames
                0x000000ee       0xa1 bss.o
 .debug_pubnames
                0x0000018f       0x61 data.o
 .debug_pubnames
                0x000001f0       0x20 load_table_dest.o
 .debug_pubnames
                0x00000210       0xd3 MultiSio.o
 .debug_pubnames
                0x000002e3       0x61 Sio32MultiLoad.o

.debug_info     0x00000000    0x19e6a
 *(.debug_info)
 .debug_info    0x00000000     0x37b4 loader_main.o
 .debug_info    0x000037b4     0x34e2 sub.o
 .debug_info    0x00006c96     0x32b0 intr_table.o
 .debug_info    0x00009f46     0x3363 bss.o
 .debug_info    0x0000d2a9     0x2e72 data.o
 .debug_info    0x0001011b     0x32bc load_table_dest.o
 .debug_info    0x000133d7     0x3641 MultiSio.o
 .debug_info    0x00016a18     0x3452 Sio32MultiLoad.o

.debug_abbrev   0x00000000      0xa2a
 *(.debug_abbrev)
 .debug_abbrev  0x00000000      0x156 loader_main.o
 .debug_abbrev  0x00000156      0x16b sub.o
 .debug_abbrev  0x000002c1      0x119 intr_table.o
 .debug_abbrev  0x000003da      0x101 bss.o
 .debug_abbrev  0x000004db      0x101 data.o
 .debug_abbrev  0x000005dc      0x101 load_table_dest.o
 .debug_abbrev  0x000006dd      0x1cf MultiSio.o
 .debug_abbrev  0x000008ac      0x17e Sio32MultiLoad.o

.debug_line     0x00000000      0xe82
 *(.debug_line)
 .debug_line    0x00000000      0x3d7 loader_main.o
 .debug_line    0x000003d7      0x1cd sub.o
 .debug_line    0x000005a4      0x4d0 MultiSio.o
 .debug_line    0x00000a74      0x40e Sio32MultiLoad.o

.debug_frame
 *(.debug_frame)

.debug_str
 *(.debug_str)

.debug_loc
 *(.debug_loc)

.debug_macinfo
 *(.debug_macinfo)

.debug_weaknames
 *(.debug_weaknames)

.debug_funcnames
 *(.debug_funcnames)

.debug_typenames
 *(.debug_typenames)

.debug_varnames
 *(.debug_varnames)

.stack          0x00080000        0x0
                0x00080000                _stack=.
 *(.stack)
OUTPUT(loader.elf elf32-littlearm)
